:1000000000308A00582900000A108A100A1182075D
:1000100028340C34013406340A108A100A1182077D
:100020006F347434613463346B3479343A34253446
:100030006C34753420346F3474342F346D34693437
:100040006E34203420340034323084000008031928
:1000500038280130A100A001A00B2C28A10B2B28CF
:100060004A30A000A00B322800000000800B292895
:10007000003407080F39B900380EA000F030A00591
:100080002008F03939048700061483160610000092
:10009000831206108316061083120034B608031D5F
:1000A0005328861054288614831686108312B70EA0
:1000B0003708B8003920B70E3708B80039200D309E
:1000C000A000A00B612800341430B20024200F30AF
:1000D00083168705831286108316861083120610F6
:1000E000831606108312A8012808023C031C8028EE
:1000F0000230B20024200330B8003920A80A742846
:100100000D30A000A00B82280230B80039200D303D
:10011000A000A00B8928A8012808023C031C9C28E9
:1001200028080420A900B6012908B7004E20023093
:10013000B2002420A80A8C288A119C291030A00023
:10014000A301AC01A90CA80C031CAC282A08A30726
:100150000318AC0A2B08AC07AC0CA30CA20CA10C26
:10016000A00BA2288A11B92901303202B400330849
:10017000023C031DBD284030B40734088038B50068
:10018000B6013508B7004E20003431080C3A031987
:10019000D328063A0319DB28073A0319E128053A60
:1001A0000319E628EB28B6010130B7004E200230D3
:1001B000B2002420F7280130B2000230B300B4208E
:1001C000F7280130B200B300B420F728B601103090
:1001D000B7004E20F72831081F3C031CF1280730D8
:1001E000B1050130B6003108B7004E20F7280034C1
:1001F0000408B0002A0EF038AC00AC07E23EAD00B7
:10020000323EAF002A080F39AD07AD07AF07E93E10
:10021000AE00AE07AE07290E0F39AE07AF07AE0D21
:10022000AF0DAF09AF0D29080F39AF07AC0D07307F
:10023000AB000A30AF07AE03031C1A29AE07AD03AB
:10024000031C1E29AD07AC03031C2229AC07AB031A
:10025000031C26292B3084000730300584072F30FB
:10026000040203194F290008A000031D3D29301A7C
:100270004D29B0193F29203040290830B0003030D6
:10028000A007AA010408A9002008AB002008B100BB
:10029000C520290884002B08A000840A2F29000803
:1002A000A0003030A0072008B100C5208A11D8294D
:1002B00084011F30830583161F149F141F159F117F
:1002C000FF308312A50083161F149F141F159F1162
:1002D00083121F109412A51225088316870083121B
:1002E00025162508831687008312A5112508831675
:1002F0008700003083129400831694000108C739E8
:10030000383881009730831290000030A1009200AD
:10031000003083169200831225112508831687006A
:10032000831207110C309700A51425088316870047
:1003300083129D019D0164288F018E010230A80067
:10034000FA30B2002420A80BA0290F08A3000E0841
:10035000A0000F082302031DA5292008A6002308DA
:10036000A7002708A9002608A800AB012830AA008A
:100370009E282208A7002108A6002608A00027081A
:10038000A300C2290230B200B300B420A80128089B
:100390000C20A80AA000B100C52007302802031DC8
:1003A000C729103084002708AA002608A900F828C9
:1003B0000A30A90029080C20A90AA000B100C52014
:0C03C00013302902031DDA299C29630078
:02400E00793FF8
:00000001FF
